:100000000C9494020C94CC020C94CC020C94CC0270
:100010000C94CC020C94CC020C94CC020C94CC0228
:100020000C94CC020C94CC020C94A2240C94742555
:100030000C94B41F0C94CC020C94CC020C94CC0203
:100040000C94CC020C94CC020C94CC020C94CC02F8
:100050000C94CC020C943C200C94CC020C94CC025A
:100060000C94CC020C94CC020C94CC020C94CC02D8
:100070000C94CC020C94CC020C94CC020C94CC02C8
:100080000C94CC020C94CC020C94CC020C94CC02B8
:100090000C94CC020C94CC020C94CC020C94CC02A8
:1000A0000C94CC020C94CC020C94CC028F058F05DE
:1000B000BB05BB0523064E074E074E074106DA0671
:1000C000EB06EB06E1250826002708260027542624
:1000D00077260027CE26DD2629001E001F002000DF
:1000E00021002200230024002500260027002D00E7
:1000F0002E002A002A004C002B0014001A000800D1
:10010000150017001C0018000C00120013002F002F
:1001100030003100000049003900040016000700DB
:1001200009000A000B000D000E000F003300340020
:100130000000280000004B00E1002C001D001B0007
:1001400006001900050011001000360037003800C5
:10015000E500520000004E00E000E300E200000075
:100160002C0000002C0000002C000000E6000151D3
:100170005000510000004F00005C3A003B003C0082
:100180003D003E003F00400041004200430044006B
:1001900045000100010001000100C35CC45CC65CB5
:1001A000C75CC85CC95CCA5CCB5C01000100010093
:1001B0000100010000000100010001000100010038
:1001C0000100010001000100010001000100010027
:1001D0000000010000000100010001000100010019
:1001E000C05CBE5CBF5CC15C01000100010001009D
:1001F00001000100000001000100010001000000F9
:1002000001000000010000000100000001000100E9
:10021000010001000000010000047F3F1F64321450
:10022000643214783C1E1E140A0522232526282930
:100230002A2C2D2F3032333536383A3B3D3E404262
:10024000434547494A4C4E5051535557595A5C5EA5
:100250006062646668696B6D6F71737577797B7DB9
:100260007F81838587898A8C8E90929496989A9CB8
:100270009E9FA1A3A5A7A8AAACAEAFB1B3B4B6B8D0
:10028000B9BBBCBEBFC1C2C3C5C6C7C9CACBCCCD32
:10029000CED0D1D2D2D3D4D5D6D7D7D8D9D9DADA0D
:1002A000DBDBDBDCDCDCDCDCDDDDDDDDDCDCDCDC8D
:1002B000DCDBDBDBDADAD9D9D8D7D7D6D5D4D3D2C1
:1002C000D2D1D0CECDCCCBCAC9C7C6C5C3C2C1BF9F
:1002D000BEBCBBB9B8B6B4B3B1AFAEACAAA8A7A503
:1002E000A3A19F9E9C9A98969492908E8C8A8987BF
:1002F0008583817F7D7B79777573716F6D6B69689D
:10030000666462605E5C5A5957555351504E4C4A70
:100310004947454342403E3D3B3A3836353332301B
:100320002F2D2C2A292826252322FFAA7F5540007D
:1003300001010101010101010102020202020202A6
:100340000202030303030303030304040404040479
:10035000040505050505060606060607070707073F
:1003600008080808090909090A0A0A0B0B0B0C0CF2
:100370000C0D0D0D0E0E0E0F0F0F1010111111128E
:100380001213131414151516161717181819191A0D
:100390001A1B1B1C1D1D1E1E1F2020212222232470
:1003A00024252626272829292A2B2C2D2D2E2F30AF
:1003B000313232333435363738393A3B3C3D3E3FC3
:1003C000404142434445464748494A4C4D4E4F50B0
:1003D000515354555658595A5B5D5E5F616264656E
:1003E0006668696B6C6D6F7072737577787A7B7DF8
:1003F0007E8082838587888A8C8E8F91939596984C
:100400009A9C9EA0A2A3A5A7A9ABADAFB1B3B5B767
:10041000BABCBEC0C2C4C6C9CBCDCFD1D4D6D8DB3E
:10042000DDDFE2E4E7E9EBEEF0F3F5F8FAFDFF22B9
:10043000034B006500790020003600350020005590
:10044000006E006900760065007200730061006C48
:10045000000000100346006F00780020004C00618F
:1004600000620000000403090409023B00020100CD
:10047000A0FA090400000103010100092111010093
:100480000122400007058103080001090401000161
:10049000030000000921110100012232000705823A
:1004A0000320000112010002000000084C46040075
:1004B00001000102000105010980A1018503190164
:1004C0002AB700150126B700950175108100C005F7
:1004D0000C0901A101850419012AA002150126A019
:1004E00002950175108100C005010906A1010507EB
:1004F00019E029E71500250195087501810295018C
:10050000750881010507190029FF150026FF0095D0
:1005100006750881000508190129059505750191E1
:1005200002950175039101C011241FBECFEFDAE0DF
:10053000DEBFCDBF04B603FE18C08091C602909105
:10054000C702A091C802B091C9028730904BA74062
:10055000B04B59F41092C6021092C7021092C80212
:100560001092C902E0E0F8E3099511E0A0E0B1E0E3
:10057000E6E8F0E502C005900D92A03CB107D9F77E
:1005800022E0A0ECB1E001C01D92A63CB207E1F769
:100590000E944C130C9441280C94000081E00895B3
:1005A00081E008950C94D00208950C94D4021F9316
:1005B000CF93DF9300D000D01F92CDB7DEB7498331
:1005C0005A836B833091C30189819A81311114C0A0
:1005D000662359F0222349F00E948709182F682FBB
:1005E00089819A810E94300903C00E945B09182FFB
:1005F00069817A81812F04C00E94870969817A818B
:100600000F900F900F900F900F90DF91CF911F914F
:100610000C94B510FC01262F4081518162817381B9
:1006200084810C94D70281E00895CF93DF93EC018D
:1006300060E00E940A03BE01DF91CF910C94D502C5
:100640000C94FD110C94F91108950E94DA070E9490
:1006500024032FEF84E39CE0215080409040E1F799
:1006600000C000000C9462200F931F93CF93DF9380
:100670008C0161E00E940A03EC01B8010E94D202E1
:10068000882309F44BC0B801CE010E947B1B88234C
:1006900009F444C0B801CE010E948D1E8823F1F1F7
:1006A000B801CE010E94A11C8823C1F1B801CE017E
:1006B0000E94E91D882391F1B801CE010E94BF1963
:1006C000882361F1F8018281882309F1CB358DE51A
:1006D000D807C1F050F4C115FCE5DF0781F0CF3D2C
:1006E000DC45A9F40E94BE0E19C0CC35EDE5DE074D
:1006F00061F0CD35DD4559F40E94010E08C00E941D
:1007000025030CC00E940A0E02C00E940D0EC801F3
:10071000DF91CF911F910F910C94CE0280E0DF9179
:10072000CF911F910F9108950E94961F80E00E9423
:10073000B01B0E94C3030C943C180E949F1A0E9495
:10074000C6030E9408190C949C1F08950C94A503DD
:1007500081E00895CF93C82F0E94A803882329F031
:10076000C2FD02C0769A01C07698CF9108956E9A24
:10077000769A0895CF93C82F0E94A6038C2F0E94CB
:10078000AA03CF91089580E00C94BA030E94E91E59
:100790000C94BA030E94E91E9091C201891721F0BE
:1007A0008093C2010C94BA030895CF93DF93CDB721
:1007B000DEB72B970FB6F894DEBF0FBECDBF4F83C9
:1007C000588769877A878B8761110E944D0D9E013A
:1007D0002F5F3F4F86E0F90111928A95E9F785E096
:1007E000FE013796D90101900D928A95E1F7898132
:1007F0009A814C815D81452B31F09F3F31F491E02E
:100800008F3F19F403C091E001C090E090FF09C050
:1008100049815A816B817C818D819E810E946E0C01
:1008200005C0C9010E9413038111F2CF2B960FB6A8
:10083000F894DEBF0FBECDBFDF91CF910895FC01CC
:10084000808191810E94C9090895CF93882309F47A
:100850009CC0C82F8238C1F40E94E91E81FD95C05A
:1008600069E380910201909103010E946E1F0E9432
:100870006F0D2FEF81EE94E0215080409040E1F722
:1008800000C0000069E319C0833801F50E94E91E29
:1008900080FD7BC063E580910201909103010E947D
:1008A0006E1F0E946F0D2FEF81EE94E0215080406B
:1008B0009040E1F700C0000063E580910201909153
:1008C00003010E94701FCF910C946F0D8438C1F406
:1008D0000E94E91E82FD59C067E480910201909157
:1008E00003010E946E1F0E946F0D2FEF81EE94E0B6
:1008F000215080409040E1F700C0000067E4DDCF68
:100900008CEF8C0F813AD0F46C2F80910201909182
:1009100003010E94381F882349F06C2F8091020147
:10092000909103010E94701F0E946F0D6C2F8091A7
:100930000201909103010E946E1FC5CF80E28C0FCF
:10094000883048F4C77081E001C0880FCA95EAF783
:100950000E94300DB8CFEBE5EC0FE33040F4F0E04F
:10096000EE5AFE4F808190E0CF910C94001FC85A40
:10097000C73158F4EC2FF0E0EE0FFF1FEC5DFE4F97
:1009800080819181CF910C94161FCF910895882377
:1009900009F45BC0682F823879F40E94E91E81FF58
:1009A00054C069E380910201909103010E946E1F7F
:1009B0000E946F0D69E310C08338B1F40E94E91EF4
:1009C00080FF43C063E580910201909103010E9482
:1009D0006E1F0E946F0D63E58091020190910301EB
:1009E0000E94701F0C946F0D843879F40E94E91EE8
:1009F00082FF2BC067E480910201909103010E9465
:100A00006E1F0E946F0D67E4E7CF8CEF860F813A6F
:100A100018F380E2860F883048F4677081E001C0E7
:100A2000880F6A95EAF70E94360DDCCF8BE5860FBA
:100A3000833020F480E090E00C94001F685A673106
:100A400020F480E090E00C94161F08951F93CF933C
:100A5000DF93182FEB010E942504209741F08FE9C6
:100A60009FE00197F1F700C000002197F6CF812F9A
:100A7000DF91CF911F910C94C704893319F060E086
:100A800070E002C060E570E00C942605882321F038
:100A90000E94300D0C946F0D0895882321F00E9460
:100AA000360D0C946F0D0895CF92DF92EF92FF9266
:100AB0000F931F93CF93DF937C01D62FC72FFC0199
:100AC0001281058102950F700E94260D8823B9F0CE
:100AD0001123A9F08C2F807F803421F080E28D0FCC
:100AE000883068F08091880282FD09C082E00E940F
:100AF000CF0D0E94260D91E0D82ED92601C0D12C11
:100B0000CC2EC2948FE0C8228C2D90E08C309105C1
:100B100008F0C4C1FC01EA5AFF4F0C949C278C2FAB
:100B2000807FCF70882311F0C295C07F112399F088
:100B3000CC2309F49FC180E28D0F883010F0D111D1
:100B400004C08C2F0E94300D03C08C2F0E94400DDA
:100B50000E946F0D8FC18D2F0E94C704CC2309F412
:100B60009DC180E28D0F883038F1DD2329F18C2F73
:100B70000E94460D24C08C2F807FCF70803211F0F0
:100B8000C295C07FDD2319F0D130A1F13DC0809125
:100B9000880282FF17C0112349F0CC2329F08C2F43
:100BA0000E94300D0E946F0D80E065C180E00E94C0
:100BB000C704CC2309F472C18C2F0E94360D0E9409
:100BC0006F0D6CC1112371F0002341F0013031F43D
:100BD0000E94500D8C2B0E94580D60C10E94500D38
:100BE0008C2B1DC0002319F0013009F457C10E945D
:100BF000650D25C0112321F0063008F04FC10EC04D
:100C0000053008F04BC11BC0112361F0002331F007
:100C1000F701858180FF2EC18F7085838C2F0E9404
:100C200046053CC1002359F0D93309F034C1FFEF28
:100C300007EE13E0F15000401040E1F72AC18C2F7D
:100C40000E944D052BC18C2F86958695837019F0D7
:100C5000813061F023C1112321F08D2F9C2F9370DF
:100C600002C080E090E00E94001F20C1112321F00B
:100C70008D2F9C2F937002C080E090E00E94161F81
:100C800015C18C2F837009F047C011110BC12D2F96
:100C9000229526952770220F220F6D2F6F70862FB9
:100CA00090E0A0E0B0E0022E04C0880F991FAA1FB8
:100CB000BB1F0A94D2F7D4FF10C04FE050E060E0B1
:100CC00070E004C0440F551F661F771F2A95D2F7A6
:100CD000409550956095709503C040E050E0BA0192
:100CE000C695C695C3708A019B01082B192B2A2B28
:100CF0003B2BC901B801C23049F058F4C13019F09A
:100D00000E944608CFC00E943408CCC00E945808F8
:100D1000C9C00E943208C6C0112319F08C2F8170FF
:100D200001C08695882309F4BDC02D2F22952695F4
:100D30002770220F220F6D2F6F70862F90E0A0E09A
:100D4000B0E0022E04C0880F991FAA1FBB1F0A948F
:100D5000D2F7D4FF10C04FE050E060E070E004C074
:100D6000440F551F661F771F2A95D2F7409550955F
:100D70006095709503C040E050E0BA01C695C695F5
:100D8000C3708A019B01082B192B2A2B3B2BC9010D
:100D9000B801C23049F058F4C13019F00E940B0973
:100DA00081C00E94F9087EC00E941D097BC00E947C
:100DB0006C0878C0CF70112339F08C2F0E949208F4
:100DC0008D2F0E9446056EC08D2F0E944D058C2FE1
:100DD0000E94B30867C0D23F21F128F4D03F41F010
:100DE000D13FC1F043C0D33F19F1D43F79F03EC0A9
:100DF000112341F0053008F051C08C2F8F710E94F3
:100E0000D8084CC0063008F049C0F7CF809188025E
:100E100082FF18C0112339F08C2F8F710E94920825
:100E20003DC01123C9F38C2F8F710E94B30836C0C7
:100E3000112329F08C2F8F710E947D082FC00E94F2
:100E400078082CC0112349F0CF718C2F0E94920892
:100E500063E08C2F0E94B40D21C081E00E94CF0D71
:100E60000230E0F082E00E94CF0D18C0112331F073
:100E7000002391F28D2F0E94250410C0002399F2C7
:100E8000D93349F41FEF27EE33E0115020403040B2
:100E9000E1F700C000008D2F0E94C70488EF8C0D81
:100EA000843020F40E94E91E0E94BA03DD20C9F0BC
:100EB0000E94220D80FD15C0F70112820E941C0DB8
:100EC0000E949208C7010E9492070E941C0DDF91A8
:100ED000CF911F910F91FF90EF90DF90CF900C94E6
:100EE000B308DF91CF911F910F91FF90EF90DF90AA
:100EF000CF9008950F931F93CF93DF93EC016881F8
:100F000079818A810E94D4098C010E942F090E9454
:100F10002008B801CE010E945405DF91CF911F91A6
:100F20000F910895CF93DF93EC01988189812B81F4
:100F30003C81232B31F08F3F31F481E09F3F19F446
:100F400003C081E001C080E080FD1DC0CE010E9491
:100F50003403811110C00E94260D8823A1F08A81DC
:100F6000882389F08091880282FD0DC082E0DF91A4
:100F7000CF910C94CF0DCE010E947A07CE01DF9164
:100F8000CF910C941503DF91CF91089580E090E00C
:100F90000E94001F80E090E00E94161F0E944D0DED
:100FA0000C946F0D80910201909103010E94721FB9
:100FB0000C94C6070E943D0D0C94D20792959F7029
:100FC000963079F010F4925001C09A50923068F443
:100FD000803F69F018F4883E40F409C0843F29F44A
:100FE00006C0883E20F0813F11F080E0089581E046
:100FF0000895FC01808191810E94C9090E94DE0749
:101000000895CF93DF9300D000D01F92CDB7DEB705
:101010000F900F900F900F900F90DF91CF91089548
:10102000CF93DF9300D000D000D0CDB7DEB72696A7
:101030000FB6F894DEBF0FBECDBFDF91CF910895FC
:10104000089508950C9421080C9422080E94240805
:101050006093FA017093FB018093FC019093FD0172
:101060000C94C6070C9426080F931F930091FA0165
:101070001091FB012091FC013091FD01602B712B3F
:10108000822B932B1F910F910C9426080F931F9383
:101090000091FA011091FB012091FC013091FD01BA
:1010A00060237123822393231F910F910C942608B0
:1010B0000F931F930091FA011091FB012091FC0105
:1010C0003091FD0160277127822793271F910F918F
:1010D0000C9426080C9421080E946A086093F6017B
:1010E0007093F7018093F8019093F9010C94C6076F
:1010F00060E070E0CB010C946C080F931F9341E00B
:1011000050E060E070E08A019B0104C0000F111FF5
:10111000221F331F8A95D2F7C901B8011F910F9181
:101120000C946C080F931F9341E050E060E070E076
:1011300004C0440F551F661F771F8A95D2F7809110
:10114000F6019091F701A091F801B091F9018A019F
:101150009B01082B192B2A2B3B2BC901B8011F918E
:101160000F910C946C080F931F9341E050E060E0E6
:1011700070E004C0440F551F661F771F8A95D2F791
:1011800040955095609570958091F6019091F7018A
:10119000A091F801B091F9018A019B01082319235C
:1011A0002A233B23C901B8011F910F910C946C08AD
:1011B0000F931F9341E050E060E070E004C0440FE3
:1011C000551F661F771F8A95D2F78091F60190917F
:1011D000F701A091F801B091F9018A019B0108275C
:1011E00019272A273B27C901B8011F910F910C9499
:1011F0006C080F931F930091F6011091F701209155
:10120000F8013091F901602B712B822B932B1F91E8
:101210000F910C946C080F931F930091F60110919D
:10122000F7012091F8013091F901602371238223A5
:1012300093231F910F910C946C080F931F930091AF
:10124000F6011091F7012091F8013091F901602722
:101250007127822793271F910F910C946C08089592
:1012600020E1929F800D1124E82FE695E695E69502
:10127000877051E001C0550F8A95EAF785E0E89F35
:10128000F0011124EC53FE4F20E030E070E040818B
:10129000CB01022E02C0969587950A94E2F78170E1
:1012A000819584278523842781932F5F3F4F2530A5
:1012B000310569F7089520E1929F800D1124682F70
:1012C000669566956695982F977085E0689FB00142
:1012D000112440E050E080E0FB01E40FF51FEC53E7
:1012E000FE4F208130E0092E02C0369527950A94E2
:1012F000E2F721703327042E01C0220F0A94EAF787
:10130000822B4F5F5F4F4530510531F70895BF92F3
:10131000CF92DF92EF92FF920F931F93CF93DF93C1
:101320008C01C090F601D090F701E090F801F090A8
:10133000F9018091FA019091FB01A091FC01B0911B
:10134000FD01C82AD92AEA2AFB2ACFE1D0E0D70139
:10135000C6010C2E04C0B695A795979587950A945B
:10136000D2F780FD04C0219790F7B12C07C0BC2EA6
:10137000B8018C2F0E94CA100197A9F38B2DDF9121
:10138000CF911F910F91FF90EF90DF90CF90BF9082
:101390000895CF93DF93EC010E948709BE010E945C
:1013A000CA10DF91CF9108951F93CF93DF93EB0184
:1013B0009091C301992321F0CB010E94C90913C068
:1013C000882349F0CB010E948709182F682FCE018E
:1013D0000E94300904C0CB010E945B09182FBE0196
:1013E000812F0E94CA10DF91CF911F9108951F9302
:1013F000CF93DF93C091FE0116E08091FF01C817E3
:1014000099F0D0E01C9FF0011D9FF00D1124E050D9
:10141000FE4F4081518162817381848195810E9458
:1014200010082196C770E9CFDF91CF911F910895E1
:10143000409130025091310260913202709133023A
:1014400080913402909135020C941008EF92FF9233
:101450000F931F93CF93DF938091350282958F7006
:1014600009F065C080913202882309F460C0809140
:10147000FE01F090FF011091300200913102609165
:1014800033027091340291E01F3F09F090E0C09167
:101490000001D0910101292F96E0E92E8F1509F462
:1014A00046C06115710521F00F3F21F030E003C007
:1014B00031E001C0322F90E030FD36C0E89EF001EF
:1014C000E99EF00D1124DF01A050BE4F11963C9112
:1014D0001197301329C03C91311326C012963C91CC
:1014E0001297311121C013964D915C911497461BB0
:1014F000570B4C175D07C0F4809135028F708061E7
:1015000080933502EB5FFD4F80818F708061808317
:1015100080E392E00E949207DF91CF911F910F919B
:10152000FF90EF900C94F70901968770B7CFDF9189
:10153000CF911F910F91FF90EF9008959F92AF92DE
:10154000BF92CF92DF92EF92FF920F931F93CF93B0
:10155000DF93CDB7DEB761970FB6F894DEBF0FBE4D
:10156000CDBF8C0185E0F801DE011D9601900D9242
:101570008A95E1F7D8011296EC9090913002E091B3
:10158000310220913302309134022115310531F0BE
:10159000EF3F31F481E09F3F19F403C081E001C0C7
:1015A00080E0B82FB1709B2E80FD47C1D8014C91CF
:1015B00011965C9111971396AD90BC90149780E3AF
:1015C000C82E82E0D82EF0903202B501621B730B58
:1015D0002091000130910101FF2009F4D9C08091D0
:1015E00035026217730708F095C0282F207F09F095
:1015F00052C05E1313C0491311C0FE2CE1100EC07F
:101600008F708061809335020E94180AC6010E9483
:10161000920780913502F80185834DC1AB2831F0E6
:101620005F3F31F481E04F3F19F403C081E001C016
:1016300080E080FD03C081E08E2502C080E090E064
:10164000F82FF170FF2E80FF1CC08091FE012091C9
:10165000FF0136E0821709F40BC190E0389FF001DA
:10166000399FF00D1124E050FE4F6181561306C0E2
:101670006081461303C06281E61203C00196877041
:10168000E9CFFE2CEE2009F416C18091350281606D
:101690008093350254C05E1306C0491304C0E110A4
:1016A00002C0F80199C0C8010E94F907882361F1BE
:1016B000EE2051F120913502822F82958F7090E0BB
:1016C000029774F0809130029091310298878F8355
:1016D0001986BB86AA862C87CE0107960E949207A0
:1016E00086E0F801A0E3B2E001900D928A95E1F75F
:1016F0000E94260A0E94180A0AC05E1711F1C8014A
:101700000E94F90781112CC0C8010E949207FF2492
:10171000F394D1C0282F207F81F77A2DB98AA88A27
:101720006E2D89890E94010880E392E00E94920751
:1017300086E0D6011D928A95E9F70E94180AF12CDD
:10174000BAC04913DCCFE110DACFF8018583C801B4
:101750000E94920786E0D6011D928A95E9F7ABC0F8
:10176000EE2091F220913502822F82958F7090E0C9
:1017700002970CF4B5CF80913002909131029A8398
:1017800089831B82BD82AC822E83CE010196A6CFB7
:101790006217730708F044C0FE2CEE2009F4B4CFA2
:1017A0005E1330C049132EC02091350220FD21C0A8
:1017B000822F82958F70482F50E041155105C9F056
:1017C000F80125834F30510541F08F5F982F929596
:1017D000907F822F8F70892B8583C8010E9492078A
:1017E00086E0F801A0E3B2E001900D928A95E1F75E
:1017F0003CC086E0F801A0E3B2E001900D928A952A
:10180000E1F759C0C8010E94F907811169CF8091A1
:101810003502816080933502C8010E9492074BC057
:101820007A2DB98AA88A6E2D89890E94010886E0DE
:10183000D6011D928A95E9F718C0EE2009F464CF0D
:10184000C8010E94F907F82E882309F45DCF86E0CD
:10185000F801A0E3B2E001900D928A95E1F780E3F0
:1018600092E00E941F040E94260A0E94180A23C0C8
:101870004D875E878D859E850E94C909292F2295F7
:101880002F70223028F49F7039F0811105C00BC0F1
:10189000243028F49F7049F4805E883020F0C8011D
:1018A0000E9492079F2CF92C06C0D80115969C9196
:1018B000907F91F7F8CF8F2D61960FB6F894DEBF29
:1018C0000FBECDBFDF91CF911F910F91FF90EF9091
:1018D000DF90CF90BF90AF909F9008951F93CF93CC
:1018E000DF93CDB7DEB72C970FB6F894DEBF0FBEEF
:1018F000CDBF4F83588769877A878B879C87CE01B6
:1019000007960E949E0A8823D1F09F8188852A85A8
:101910003B85232B31F08F3F31F481E09F3F19F459
:1019200003C081E001C080E080FD47C04F81588541
:1019300069857A858B859C850E9410083EC086E06B
:10194000FE013796DE01119601900D928A95E1F71E
:10195000FF81E8856A857B856115710531F0EF3F70
:1019600031F481E0FF3F19F403C081E001C080E061
:1019700080FD23C02091FF0130E0C90101968770EE
:1019800099274091FE0150E084179507F1F1F98302
:10199000EA837D836C8396E0929FD001939FB00D84
:1019A0001124A050BE4FFE01319601900D929A95E0
:1019B000E1F78093FF010E94F70916E08091FE0194
:1019C0009091FF01891771F1189FC0011124805077
:1019D0009E4F0E949E0A882329F1E091FE011E9FDE
:1019E000F0011124E050FE4F4081518162817381EA
:1019F000848195810E9410088091FE0190E00196FB
:101A0000877099278093FE01D9CF0E94DA07109240
:101A1000FF011092FE01E0E3F2E086E0DF011D929B
:101A20008A95E9F72C960FB6F894DEBF0FBECDBFAE
:101A3000DF91CF911F91089580913E028595859504
:101A40008595089580913E028770089590913E0299
:101A5000977081E009F480E008958091490208952B
:101A600090914902892B8093490208958095909125
:101A700049028923809349020895109249020895EA
:101A800090914802892B8093480208958095909107
:101A900048028923809348020895109248020895CD
:101AA00080913F02089508950C94530D0C94540DA9
:101AB0009091880292FD08C090913F02981721F002
:101AC00080933F020C94560D089580913F02882325
:101AD00029F010923F0280E00C94560D0895CF93A8
:101AE000DF93E0910201F09103018091490280832C
:101AF000E0910201F0910301908180914802892BCD
:101B0000808380913F02882381F0E0910201F0916F
:101B100003019081892B80838091020190910301C0
:101B20000E942C1F81110E94650DC0910201D0916D
:101B3000030148E050E066E372E0CE010E94EC272A
:101B4000892B69F088E0FE01A6E3B2E001900D92D6
:101B50008A95E1F7CE01DF91CF910C94F51EDF91CC
:101B6000CF9108950C94530D9091880292FD10C06E
:101B700098E0899F90011124262B20933E020E9419
:101B8000920880913E028595859585950C94B20DBD
:101B90000C94920810923E0280E00C94B20D2091B9
:101BA0003E028095822380933E02982F977099F48D
:101BB00030E0482F082E000C550B2417350759F03C
:101BC0009091880292FD07C08595859585950E9424
:101BD000B3080C94CA0D08959091880292FB2227B5
:101BE00020F9281769F080FB92F990938802809180
:101BF0008702909188020E943A0E82E00C94CF0DE9
:101C000008958091880282FB882780F991E08927D6
:101C10000C94EC0D81E00C94EC0D80E00C94EC0D38
:101C20006FEF7FEF80E090E00C942B2880E090E055
:101C30000E94072821E0893E9E4F09F020E0822F74
:101C4000089582E090E00C94F92783E090E00C94F2
:101C5000F927CF9384E090E00E94F927C82F82E211
:101C600090E00E94F9272C2F30E0A901582BCA01DF
:101C7000CF910895CF93C92F682F84E090E00E9400
:101C80000D286C2F82E290E0CF910C940D28AB01CF
:101C9000BC018FE090E00C941F28AB01BC0183E1F4
:101CA00090E00C941F2860E070E0CB010C944D0E86
:101CB00060E070E0CB010E94470E0C94530E69EE79
:101CC0007EEF80E090E00E942B2860E082E090E0D0
:101CD0000E940D2860E083E090E00E940D281092A1
:101CE000FA011092FB011092FC011092FD0160E0DC
:101CF00084E090E00E940D2860E082E290E00E9483
:101D00000D2860E085E090E00E940D2860E086E00C
:101D100090E00E940D286FEF87E090E00E940D2870
:101D200040E050E0BA0188E090E00E941F2860E0A7
:101D30008DE090E00E940D2840E050E0BA0188E17B
:101D400090E00E941F2860E087E190E00E940D284B
:101D500040E050E0BA018CE190E00E941F2860E072
:101D600070E080E290E00E942B2840E050E0BA0151
:101D700088E190E00E941F280C94580E0C945F0E8E
:101D8000682F8EE090E00C940D280E942120609333
:101D900058027093590280935A0290935B026093A9
:101DA00054027093550280935602909357020895FF
:101DB00085B7806885BF85B7806885BF089581E055
:101DC00008950C94DF0E08950C94E30E0C94E30E2A
:101DD0000C94E60E0C94E30E0C94EA0E0C94E30EB5
:101DE0000E94D80E86EA91E10E94DF1E0E94EE0E4C
:101DF0000C94EC0E0E94E40E0C94E30E0E94C011B1
:101E00000E94B7030C94661C0E940C200E94A5122D
:101E10000E94FE0E0E949F1A0E94CD180C94E80E9C
:101E20005F926F927F928F929F92AF92BF92CF926A
:101E3000DF92EF92FF920F931F93CF93DF93CDB773
:101E4000DEB72A970FB6F894DEBF0FBECDBF0E9453
:101E5000BA12C82E81110E94C50E3AE4832E32E0D8
:101E6000932E00E010E0502E802F0E94E4115C01C0
:101E7000F401619071904F01682679266114710414
:101E8000B1F40F5F1F4F0530110569F78FEF89839C
:101E90008A831B820E9415208160782F9D838C830A
:101EA00049815A816B818D810E94D5033AC080910E
:101EB0005C0281FD0E94ED11D12CEE24E394F12C03
:101EC000C3018E219F21892B29F10E94E10E8823D5
:101ED000A9F0DE825F82AE20BF2081E0AB2809F44A
:101EE00080E088870E9415208160782F9A878987F3
:101EF0004E815F8168858A850E94D503000F111F7E
:101F0000F801E65BFD4F80819181E826F926F18298
:101F1000E08207C0D394EE0CFF1CF0E1DF12D0CFBB
:101F2000B0CF81E0C11001C080E02A960FB6F894CE
:101F3000DEBF0FBECDBFDF91CF911F910F91FF90FC
:101F4000EF90DF90CF90BF90AF909F908F907F9059
:101F50006F905F9008950E94100F0E9411190E94C7
:101F6000651C0C94CA03CF93DF930E94CF10EC0141
:101F7000811522E59207E8F5811531E5930708F010
:101F8000B6C0883E910528F5803E910508F0E9C06D
:101F9000883A910570F4853A910508F07AC081304D
:101FA000910509F473C008F4D9C0049708F0D9C0AA
:101FB000D5C08F3B910508F0D1C0C85AD0E0CC0FF6
:101FC000DD1FCB5ADE4F0990D881C02DCE0194641D
:101FD000C9C0811540E5940708F069C0811550E437
:101FE000950708F060C09A9581159F4108F4B9C023
:101FF000B5C0811536E5930728F5811545E59407A9
:1020000008F092C0811554E5950708F087C0AC012F
:1020100043705527282F26952695C115D34508F0DE
:102020006CC081E090E002C0880F991F4A95E2F7EA
:1020300040E2249F90011124EC01C22BD32BCE014E
:102040009C6890C081152AE5920780F4811539E5D6
:10205000930708F072C0811548E5940708F47EC024
:10206000D82FCC27CE01806F906A7CC09056811506
:10207000904208F073C08D2F8F710E946311DD278D
:10208000D0628F71AE01582BCA016CC081E090E024
:1020900069C0C55AD0E0CD57DE4F8881C82FD0E047
:1020A000CE0190645FC0DF70CE01906A5BC074E0C7
:1020B000969587957A95E1F7282F23703C2F3370FA
:1020C00081E090E002C0880F991F3A95E2F79C6882
:1020D000AC01522B9A019C2F9F709695969550E2D9
:1020E000959FE0011124C9018C2B9D2B3BC0D82F5B
:1020F000CC27CE01816F906A35C081E090E002C0AC
:10210000880F991F4A95E2F750E2259F900111240C
:10211000EC01C22BD32BCE019A6824C0D82FCC2738
:10212000CE01846F906A1EC00E9463118F7190E08F
:10213000D82FCC27CE01906215C08F700E946311FA
:1021400094E0D695C7959A95E1F7CF70D0E0DC2F53
:10215000CC27D0699E01282BC90104C080E090E003
:1021600001C0CE01DF91CF910895E72FF0E095E017
:10217000899FE00DF11D112484E0EE0FFF1F8A9569
:10218000E1F7E60FF11DEE0FFF1FE852FF4F8591BB
:10219000949108950E94B5100E94B30F089582385B
:1021A000910569F1B0F48133910509F46DC048F4EB
:1021B0008932910509F463C08A32910509F469C036
:1021C00008958533910509F455C089339105B9F017
:1021D0000895833E910569F138F4803E9105B1F090
:1021E000823E910509F10895863E9105A9F1873E49
:1021F0009105B9F1843E910509F064C023C0209196
:10220000870220FD4FC021FD4DC0089580918702B7
:1022100080FD44C08091880280FF44C08091870285
:1022200084FD42C083EE4DC08091870282FF38C09A
:10223000F5CF8091870282FD33C08091880280FDB6
:1022400031C0ECCF8091880281FF32C0809187023B
:1022500084FD2AC087EE35C08091870283FF26C0A7
:10226000F5CF8091870283FD21C08091880281FD96
:102270001FC0ECCF8091870285FD1CC01DC08091DE
:10228000870285FD19C016C08091870286FD16C0A1
:1022900017C08091870286FD13C010C089E311C06A
:1022A00082EE0FC080EE0DC080E00BC086EE09C04C
:1022B00084EE07C089E205C085E303C08AE201C05D
:1022C00081E390E008959091870292FF0DC0282F3E
:1022D0002871283019F4877F846006C0282F247164
:1022E000243011F48B7F886093FF0DC0282F287154
:1022F000283119F4877E846106C0282F2471243187
:1023000011F48B7E88612091880220FF0DC0382F48
:102310003871383019F4877F816006C0382F3171E9
:10232000313011F48E7F886021FF0DC0282F287175
:10233000283119F4877E816106C0282F217121314F
:1023400011F48E7E886194FD877E089580E0089563
:102350000C94100E0E94BA128FE39CE90197F1F7DA
:1023600000C000000E94BA1280E00E94E41180FFC9
:1023700004C00E94A8110C94622008950C94AA1124
:102380000E94160E811102C00E94BE0E0E94210EF4
:1023900080935C020E94290E9093880280938702AA
:1023A0000E94BE110E94250E682F70E080E090E030
:1023B0000E9432086091F6017091F7018091F80156
:1023C0009091F9010C946A08E82FF0E0EE0FFF1FDE
:1023D000ED56FD4F808191810895089580EA8A9598
:1023E000F1F7089500C008950C94EE1108950C942F
:1023F000F6110C94F7110C94F6110C94FB11F8944F
:10240000E82FE295EF70F0E031A1282F2F7081E0E6
:1024100090E001C0880F2A95EAF7982F90959323B2
:1024200091A392A1892B82A3789408950F931F936F
:10243000CF93DF93C6E9D1E089918F3F11F00E94DD
:10244000FF1181E0CB39D807B9F7C6E8D1E006E93A
:1024500011E089918F3F11F00E94FF110C171D07A9
:10246000C1F7DF91CF911F910F910895BF92CF9245
:10247000DF92EF92FF920F931F93CF93DF938C0124
:10248000C62FD0E0CE018A569E4F6C01FC01908190
:102490009F3F09F450C0B62EF894E92FE295EF70F3
:1024A000F0E081A19F7021E030E001C0220F9A95F9
:1024B000EAF7822B81A382A12095282322A3789476
:1024C0000E94F211E6E8F1E046E951E021E030E057
:1024D000E12CF12C61916F3F89F0A62FA295AF708E
:1024E000B0E090968C9190E06F7002C095958795C2
:1024F0006A95E2F780FD02C0C90102C080E090E069
:10250000E82AF92A220F331F4E175F0719F7F60141
:1025100080818F3F11F00E94FF1161E0E114F1040E
:1025200009F460E08B2D0E94F411CC0FDD1FC00F69
:10253000D11FF982E882DF91CF911F910F91FF9017
:10254000EF90DF90CF90BF9008950E9416128AE01E
:10255000E3E9F2E0DF01982F1D929A95E9F7E9E8A7
:10256000F2E0DF011D928A95E9F785E00E940513EC
:102570000C942003FF920F931F93CF93DF93CDB75B
:10258000DEB72A970FB6F894DEBF0FBECDBF8E011F
:102590000F5F1F4F8AE0F80111928A95E9F7F12C3D
:1025A0006F2DC8010E943612F394F5E0FF12F8CFA8
:1025B0004AE050E0B80189E892E00E94EC27FF244D
:1025C000F394009709F4F12C892B41F08AE0F8018B
:1025D000A9E8B2E001900D928A95E1F72F2D45E030
:1025E00063E972E089E892E00E9406130E942203E8
:1025F0008F2D2A960FB6F894DEBF0FBECDBFDF91A8
:10260000CF911F910F91FF9008950895FF920F931E
:102610001F93CF93DF93F82E092F162FD72FC42F98
:10262000222349F081E080935F020E94152090935D
:102630005E0280935D0280915F028823D9F08091D1
:102640005D0290915E020E942D20059798F0EF2D7B
:10265000F02FA12FBD2F80E090E04C2F50E0841789
:10266000950734F4219131912D933D930196F7CF45
:1026700010925F02DF91CF911F910F91FF9008950B
:102680000E94FA210E94040F0C9406220E940A2242
:102690000E94AB0F0C9424220E94B31F0E94E121E0
:1026A0000E94F00E0E9440130E9446130E94FA0EF0
:1026B000FBCFEF92FF920F931F93CF93DF938B018A
:1026C000682F11110AC0442329F0E82FF0E0E15DE2
:1026D000FC4F6491762F862F75C0212F30E0E82FB4
:1026E000F0E0442321F0E15DFC4FE491F0E046E0AE
:1026F000049FC0011124CFEFD0E0BE010E945227F9
:102700004BEA4603C001479F900D1124800F911D95
:10271000800F911D982F990F890FAE01421B530B0B
:102720004E9FD0014F9FB00D5E9FB00D11249B2F87
:10273000189FA0011124452F55278E01041B150B4E
:102740000E9FA0010F9F500D1E9F500D11247E0162
:10275000E81AF108E29E8001E39E100DF29E100D32
:102760001124212F3327C21BD30BCE9F9001CF9F63
:10277000300DDE9F300D112462307105A9F048F450
:102780006115710569F061307105C9F48B2F752FE2
:102790000DC06430710581F058F06630710579F430
:1027A0007E2F8B2F932F0DC0832F7B2F9E2F09C041
:1027B0008E2F7B2F952F05C08E2F732F02C07E2F5B
:1027C000852F692FDF91CF911F910F91FF90EF908F
:1027D000089541E00E945913089508950E94E91355
:1027E0000895CF93DF93762FE901682F842F0E94FD
:1027F000EE13798368838A83DF91CF910895809166
:102800009D02282F269530E02115310519F481709D
:10281000826005C02532310524F081708864809380
:102820009D02089588E090E00C940128CF92DF92F9
:10283000EF92FF926B017C010E94FF13B701A6018A
:1028400088E090E0FF90EF90DF90CF900C941F28ED
:10285000EDE9F2E083E0808311828FEF828383834E
:10286000148260817181828193810C94161480910D
:102870009D0280FF02C08695089580E008959091A2
:10288000A102933018F49F5F9093A102882351F026
:1028900060919D0270919E0280919F029091A00292
:1028A0000C941614089581E00C943F149091A102A9
:1028B000992319F091509093A102882351F06091CF
:1028C0009D0270919E0280919F029091A0020C94B3
:1028D0001614089581E00C94561470E00C94761C44
:1028E0006091080180919D0280FF0AC080910701DC
:1028F00023E0829FC00111248E559D4F0C946D14CE
:102900008091090190910A01891780F7E82FF0E082
:102910009F01220F331FE20FF31FEE55FD4F11826F
:10292000108212828F5FF0CF90919D0290FF16C0AF
:102930009091090120910A01921770F4E92FF0E0BB
:10294000DF01AA0FBB1FEA0FFB1FEE55FD4F81836E
:10295000608342839F5FF0CF0C9470140895CF93EF
:10296000DF9300D01F92CDB7DEB790919D0290FF0C
:102970000AC09E012F5F3F4F0E94F1134B81698176
:102980008A810E9494140F900F900F90DF91CF9145
:102990000895CF93DF93EC01EC81F0E0E65DFD4F0D
:1029A0004491EDE9F2E0628181810E94AF148C8153
:1029B0008F5F8C83DF91CF910895CF93DF93EC01EC
:1029C000EDE9F2E0438162818C810E94AF148C8139
:1029D0008F5F8C83DF91CF9108950F931F93CF93D7
:1029E000DF9300D01F92CDB7DEB78C0180916002DB
:1029F00081110AC09E012F5F3F4F4FEF6FEF0E9482
:102A0000F1138A8180936002F8018481813051F052
:102A100028F0823061F4409160020AC08091600227
:102A200040E007C06091600240E080E003C040E009
:102A300080E060E00E949414F801848190E00196A7
:102A400063E070E00E94662784830F900F900F90E0
:102A5000DF91CF911F910F910895AF92BF92CF92C6
:102A6000DF92EF92FF920F931F93CF93DF9300D0EB
:102A70001F92CDB7DEB7182FF62E042FE22E9091BD
:102A80009D0290FF6DC0E92FE695AE2FB0E0A556F0
:102A9000BE4F8C9180936C029E7F923061F49E01B8
:102AA0002F5F3F4F812F0E94F1134B8169818A81F3
:102AB0000E94941443C0823019F40091A0023EC0D9
:102AC000863019F410919E0239C08930D9F38931CA
:102AD000A9F5E9518E2F8170D82EE695F0E0E65DDC
:102AE000FC4FA590B490C12CBB2460910B01C6167D
:102AF00018F52C2D30E0A29EC001A39E900DB29E31
:102B0000900D112470E00E945227812FD11002C035
:102B1000860F01C0861B90910901290F311DA90163
:102B2000440F551F240F351F2E553D4F402F6F2D3D
:102B30000E94F113C394D9CF0E94701410939E0287
:102B4000F0929F020093A002EE2051F060919D024E
:102B500070919E0280919F029091A0020E94161493
:102B60000F900F900F90DF91CF911F910F91FF90D9
:102B7000EF90DF90CF90BF90AF900895EDE9F2E035
:102B80009181282F4381628188E0890F0C942D1553
:102B900081E00C94BE15EDE9F2E09181282F43818C
:102BA000628188EF890F0C942D1581E00C94CB1570
:102BB000EDE9F2E0628128E0620F08F46FEF282F60
:102BC000438181810C942D1581E00C94D815EDE999
:102BD000F2E0628128E0621B08F460E0282F438164
:102BE00081810C942D1581E00C94E715EDE9F2E05C
:102BF000438128E0420F08F44FEF282F6281818142
:102C00000C942D1581E00C94F615EDE9F2E043816A
:102C100028E0421B08F440E0282F628181810C9457
:102C20002D1581E00C94051620E00C942D15FF92D3
:102C30000F931F93CF93DF93EC01F12C0FEF10E074
:102C400060910B01F616F0F4809109012F2D30E010
:102C5000280F311DC901880F991F280F391F2E55C4
:102C60003D4F70E0C8010E946627962F8C814091ED
:102C7000A00260919F02F99E800D11240E94F11321
:102C8000F394DECF0E9470149A818C8190FF02C071
:102C90008F5F01C081508C83DF91CF911F910F9185
:102CA000FF900895AF92BF92CF92DF92EF92FF9282
:102CB0000F931F93CF93DF93FC01828180FF02C0AB
:102CC0000FEF01C001E010E046E0A42E80910B015F
:102CD000181708F043C080910901C12ED12CE601DC
:102CE000C80FD11DCE01880F991FC80FD91FCE550F
:102CF000DD4F198218821A8234E0E32EF12CB12CB8
:102D0000809162028B0D87302CF06A2D0E9444273F
:102D1000892F05C087FF03C090910B01890F082EF2
:102D2000000C990BC816D90691F48091A0028E9DD3
:102D3000A0018F9D500D11245595479555954795A8
:102D40009E0160919F0280919E020E94F113B00E3D
:102D5000F1E0EF1AF108A1F61F5FB8CF0E947014DE
:102D600080916202013031F4811102C080910B0127
:102D7000815007C090E0019660910B0170E00E94C5
:102D8000662780936202DF91CF911F910F91FF9090
:102D9000EF90DF90CF90BF90AF900895CF93809148
:102DA000090190910A01891770F4E82FF0E09F0162
:102DB000220F331FE20FF31FEE55FD4F11821082D9
:102DC00012828F5FF0CFC0E060910B01C617C0F593
:102DD000EC2FF0E070E0CF010E94662720910901FE
:102DE000820F20916102022E000C330B90E0E2175B
:102DF000F307CCF020910601022E000C330B2E17A6
:102E00003F078CF09C01220F331F820F931F9C0100
:102E10002E553D4F4091A00260919F0280919E02ED
:102E20000E94F1130BC0FC01EE0FFF1F8E0F9F1FBE
:102E3000FC01EE55FD4F118210821282CF5FC4CF8C
:102E40000E9470142091050180916102820F80938D
:102E5000610290910601920F9093060119165CF49D
:102E6000082E000C990B40910B0150E04150510984
:102E7000841795071CF0219520930501CF910895A3
:102E80008F929F92AF92BF92CF92DF92EF92FF927A
:102E90000F931F93CF93DF938C01FC014481C42FC8
:102EA000D0E09E01DE010E94AA279B01AC010E9496
:102EB000C0276B017C01E0E2F0E0EC1BFD0BA5E517
:102EC000B0E09B01AC010E94C0274B015C019F0157
:102ED000DF010E94A2279B01AC010E94CB279B012E
:102EE000AC012C0D3D1D4E1D5F1DC501B4010E949E
:102EF0007A27C22FD22F2A3228F4F3E02F9F900195
:102F000011240DC025E530E02C1B3109C901880FC3
:102F1000991F280F391F37FF02C02F5F3F4F35958C
:102F20002795C22FC095F12C85E5E82EED1A8091EA
:102F30000B01F816C8F4F1FC02C08E2D01C08D2FD4
:102F4000909109012F2D30E0290F311DA901440F67
:102F5000551F240F351F2E553D4F4C2F60919F025A
:102F60000E94F113F394E3CF0E947014F80184815E
:102F7000811102C091E003C0803219F49FEF909359
:102F8000040190910401890FF8018483DF91CF91AE
:102F90001F910F91FF90EF90DF90CF90BF90AF9077
:102FA0009F908F9008950F931F93CF93DF93EC0121
:102FB00000E010E080910B01282F30E0021713078A
:102FC00024F5909109019801290F311DA901440FA1
:102FD000551F240F351F2E553D4F869590E04C818F
:102FE000081719071CF4442331F002C0411103C033
:102FF0004091A00201C040E060919F0280919E023A
:103000000E94F1130F5F1F4FD5CF0E9470148C8167
:1030100090E00196817099278C83DF91CF911F9169
:103020000F910895EDE9F2E080818E7F80836081C9
:103030007181828193810E94161410926D022FEF8C
:1030400080E792E0215080409040E1F700C000000E
:103050000C947014EDE9F2E080818E7F80831092F1
:103060006D022FEF80E792E0215080409040E1F721
:1030700000C000000C94701410926D0280916A02DE
:1030800081110AC081E080936A0280919D02817063
:10309000809369020C942A18089560919D026695A8
:1030A00070E04BE050E08CE091E00E94DF27892B3C
:1030B00019F481E080936D020E94152090936402C0
:1030C00080936302089590919D0290FF35C09170A6
:1030D000811102C0926006C0853210F0986402C06F
:1030E000880F982B90939D02662351F060919D026A
:1030F00070919E0280919F029091A0020E941614EE
:1031000060919D02669570E04BE050E08CE091E0AC
:103110000E94DF27892B19F010926D0202C00E94D5
:103120004D1881E0809366024091A00260919F0259
:1031300080919E020C9414160895682F90919D0220
:10314000969581E0890F853208F081E00C94631830
:1031500081E00C949D18682F90919D0296958FEFB9
:10316000890F09F484E20C94631881E00C94AB1885
:1031700061E00C946318EDE9F2E080818160808366
:1031800086950C94B81880919D0280FD0C941218BD
:103190000C94BB1860E00C94631880916B02811151
:1031A0002EC00E94160E811104C00E94BE0E0E9405
:1031B00028140E94121460939D0270939E028093C3
:1031C0009F029093A0026E7F61F40E9428140E94D7
:1031D000121460939D0270939E0280939F029093BD
:1031E000A0020E94FF1310926D0280919D0280FF49
:1031F00003C086950E94CA1881E080936B020895EF
:10320000EDE9F2E080818160808386950C94CA1894
:1032100010926A028091690281110E9400190C9437
:103220004D180F931F93CF93DF9380916D028823E6
:1032300009F485C080916C02E0919D02E695E81B3F
:10324000E0936502823049F4F0E0EA5DFD4FE491DD
:10325000CE2FD0E009EC14E149C0863049F4F0E00B
:10326000ED5DFD4FE491CE2FD0E00DED14E13EC0B9
:10327000893051F4E695F0E0E05EFD4FE491CE2F09
:10328000D0E007E116E132C08F3051F4E695F0E06E
:10329000E35EFD4FE491CE2FD0E002E516E126C0BB
:1032A000853149F4F0E0E65EFD4FE491CE2FD0E0A9
:1032B0000EEC16E11BC0883181F0833239F4E8E16D
:1032C000F2E0C591D4910DEE14E110C0843251F4B6
:1032D000C4EFD1E003ED17E109C0C8E2D0E000E49B
:1032E00017E104C0C0EDD7E00DEE13E18091660256
:1032F000882361F0109266020E9415209093640268
:103300008093630210926802109267020E94152057
:10331000E0916302F09164028E1B9F0B8F3F9F47E9
:1033200070F4EC0FFD1FF0936402E093630283E6F8
:1033300092E0F801DF91CF911F910F910994DF91F5
:10334000CF911F910F910895882311F0FA0101C0C8
:10335000FB010994CF93DF93C82FD62F0E94371417
:103360008C1740F00E9437148D1720F4DF91CF9115
:103370000C94A8188C2FDF91CF910C94B8181F9340
:10338000CF93DF93FB0112811111C3C0EC010E94A6
:103390002D0D8272CD3CFCE5DF0709F49AC0A8F53B
:1033A000C73CECE5DE0709F476C0A8F4C43C9CE514
:1033B000D90709F45FC028F4C33CDC4509F457C0C1
:1033C00054C0C53C9CE5D90709F459C0C63CDC454E
:1033D00009F45CC04AC0CA3CFCE5DF0709F46AC0D6
:1033E00050F4C83CECE5DE0709F45AC0C93CDC45A2
:1033F00009F45BC03AC0CB3C9CE5D90709F45FC037
:10340000CC3CDC4509F460C030C0C23DFCE5DF07C0
:1034100009F46FC088F4CF3C9CE5D90709F460C07B
:1034200008F45CC0C03DFCE5DF0709F45CC0C13DA9
:10343000DC4509F45BC019C0C53D9CE5D90709F41A
:1034400060C050F4C33DFCE5DF0709F455C0C43D3E
:10345000DC4509F454C009C0C63D9CE5D90709F410
:1034600055C0CE35DD4509F454C011E052C00E946C
:10347000C3184FC045EB58E168EA78E104C048EA58
:1034800058E165EB78E10E94A41943C045ED55E190
:1034900068EC75E1F8CF48EC55E165ED75E1F3CFE7
:1034A00043EF55E164EE75E1EECF44EE55E163EF95
:1034B00075E1E9CF41E156E162E076E1E4CF42E037
:1034C00056E161E176E1DFCF4AE654E163E574E17C
:1034D000DACF43E554E16AE674E1D5CF81E017C065
:1034E00065E082E010C068E086E00DC06EE089E033
:1034F0000AC064E18FE007C067E185E104C088E1AC
:1035000006C062E289E10E94AA1903C083E20E9418
:10351000B818812FDF91CF911F91089586E090E038
:103520000C94F927682F86E090E00C940D28809188
:10353000B402847089628093B4020C94921A0E943F
:10354000160E811104C00E94BE0E0E94971A0E949E
:103550008E1A8093B402282F26952695269530E062
:103560002630310524F0877088628093B402809100
:10357000B40280FF04C086958695869501C080E0E0
:103580000C94B01B2091B402822F86958695869567
:10359000482F50E04530510554F48F5F982F990F14
:1035A000990F990F822F8770892B8093B402809195
:1035B000B40281608093B4020E94921A8091B40296
:1035C0008695869586950C94B01B8091B402982FB1
:1035D000969596959695A1F0915E990F990F990FF2
:1035E0008770892B8093B402887F91E009F490E082
:1035F0008091B40290FB80F98093B4020E94921AE9
:103600008091B4028695869586950C94B01B809126
:10361000B40280FD13C081608093B402813019F43C
:1036200089E08093B4028091B4020E94921A809142
:10363000B4028695869586950C94B01B089580916A
:10364000B40280FF08C08E7F8093B4020E94921A59
:1036500080E00C94B01B08958091B40280FD0C941E
:103660001F1B0C94071B9091B402892F8695869599
:1036700086958F5F8F719770863038F4880F880F2A
:10368000880F892B8093B40202C09093B40280917A
:10369000B402887F91E009F490E08091B40290FB3D
:1036A00080F98093B4020E94921A8091B4028695A8
:1036B000869586950C94B01B863008F085E0909135
:1036C000B4029770282F220F220F220F922B909373
:1036D000B402987F21E009F420E09091B40220FB2D
:1036E00090F99093B4020C94B01B0E945C1B8091E3
:1036F000B4020C94921A9C01FB018281882349F147
:103700002E3BFCE53F07C9F040F42C3BECE53E07BF
:1037100069F02D3B3C4561F00895203C9CE539075C
:1037200091F070F0213C3C4589F0089585E001C09E
:1037300080E00E94751B80E008950E94E51AFBCF8F
:103740000E94C21AF8CF0E942C1BF5CF0E94331B97
:10375000F2CF81E00895279A2F9808952F98089521
:103760008F929F92AF92BF92CF92DF92EF92FF9291
:103770000F931F93CF93DF93C82F863050F481119E
:1037800009C080918000877F809380000E94AE1BDB
:1037900006C0C5E080918000886080938000A09181
:1037A0008600B09187002C2F30E00E94AA2725E0E8
:1037B00030E040E050E00E947A270027122F232FAC
:1037C000342F012F122F232F3327809186009091C1
:1037D00087006CE070E00E9452276017710730F09C
:1037E000C80169E070E00E9452275EC080918600A7
:1037F00090918700E0908600F0908700E09186002D
:10380000F0918700C6E0D0E0BE010E945227060F6B
:10381000171F211D311D4801590185E0880C991C95
:10382000AA1CBB1C8A95D1F7C701BE010E94522772
:103830006F01E12CF12CA7019601260F371F411DC6
:10384000511DC501B4010E947A2769017A01E091F6
:103850008600F0918700CA01B9010E9434279B01BC
:10386000AC01DF010E94C0279B01AC01C701B6017A
:103870000E943427DC01CB012FE0B695A7959795E0
:1038800087952A95D1F7009186001091870020E056
:1038900030E0081719072A073B0728F460918600D3
:1038A00070918700CB01BC0170938D0060938C00F8
:1038B000DF91CF911F910F91FF90EF90DF90CF900C
:1038C000BF90AF909F908F90089508950E94AB1B7A
:1038D0008AE08093800089E1809381008FEF9FEFE1
:1038E00090938700809386000C949F1A6A9A2EB159
:1038F0002B7F3EB134604FB7F894FC01CB01880FA9
:10390000991F680F791F6E0F7F1FE617F70789F061
:10391000819198E03EB9000000C087FF2EB9880F62
:10392000000000C000C000C02EB900C09A9591F7F9
:10393000ECCF4FBF8FE594E00197F1F700C0000096
:103940000895CF93DF93EC01FB018281882309F472
:103950003CC1C430FDE5DF0760F4CB3F9CE5D907EF
:1039600088F49E0122503C452431310508F02EC1D7
:1039700009C0C236EDE5DE0729F0C63AFDE5DF07EE
:1039800009F024C10E94290E909388028093870237
:10399000C1318CE5D80709F4C6C008F042C0C9306F
:1039A000ECE5DE0709F49BC000F5C5308CE5D807CF
:1039B00009F485C078F4C330ECE5DE0709F478C07B
:1039C00008F07AC0C230DC4509F0F5C0809187026A
:1039D0008160EFC0C7309CE5D90709F478C008F0D2
:1039E0007AC0809187028061E4C0CD30FCE5DF07BA
:1039F00009F487C058F4CB309CE5D90709F479C0A5
:103A000008F07BC08091870288606FC0CF30FCE5F2
:103A1000DF0709F480C008F082C080918702877FA9
:103A2000C8C0CE3F9CE5D90709F471C000F5C53187
:103A3000FCE5DF0709F485C068F4C3319CE5D907CC
:103A400009F475C008F095C00E94DA0780918702DA
:103A50008F77AFC0CC3FFCE5DF07A9F108F054C079
:103A6000CB3FDC4509F0A7C08091880240C0C2303E
:103A7000EDE5DE0709F489C058F4C1158DE5D807D6
:103A800009F45AC008F069C08091880282602FC092
:103A9000C236EDE5DE0709F47CC0C63AFDE5DF0776
:103AA00009F481C0C330DD4509F085C080E06EC0F7
:103AB0008091870282607DC08091870216C08091CC
:103AC0008702886076C08091880282604FC08091B2
:103AD000870280626EC08091870280646AC00E9403
:103AE000DA0780918702806864C0846062C0816068
:103AF0003DC0809187028E7F5CC0809187028D7F60
:103B000058C08091870216C08091880218C08091A9
:103B100088028D7F2BC0809187028F7E4AC0809162
:103B200087028F7D46C0809187028F7B42C0809143
:103B30008702877F8B7F3DC0809188028D7F8E7F3B
:103B400015C08091870282FB222720F991E09227FD
:103B500090FB82F990FB83F92CC080918802982F0A
:103B6000909591708E7F892B90FB81F980938802CC
:103B700022C00E94DA078091870287FB222720F962
:103B800091E0922790FB87F914C081E00E94C00E5B
:103B900012C08091870284FB222720F991E09227AE
:103BA00090FB84F906C080918702982F909590FB36
:103BB00080F98093870280918702909188020E9409
:103BC0003A0E0E94DA0780E001C081E0DF91CF91D8
:103BD0000895CF93DF9386319C4541F5EB010E9418
:103BE0002D0D982F8A8120910201309103018823A5
:103BF00079F09A7A81E009F480E080936E02911165
:103C000002C069E201C065E3C9010E946E1F0AC0DB
:103C100080916E02811102C069E201C065E3C901B1
:103C20000E94701F0E946F0D80E001C081E0DF9153
:103C3000CF9108950F931F93CF93DF93C42FD22F6B
:103C4000FC0182818823C9F0409371020E941520F3
:103C50009093700280936F0280E28C0F883008F09E
:103C600057C0C77081E001C0880FCA95EAF7DF919D
:103C7000CF911F910F910C944605809171024813CA
:103C800030C080916F02909170020E942D20883C7C
:103C9000910538F510E21D0FCD17B9F080E28C0FB9
:103CA000883040F4C77081E001C0880FCA95EAF7F8
:103CB0000E944D05183028F581E09D2F977001C0B6
:103CC000880F9A95EAF70E944605802F0E943D05CD
:103CD0001830F0F4D77081E001C0880FDA95EAF768
:103CE0000AC080E28C0F883098F4C77081E001C070
:103CF000880FCA95EAF7DF91CF911F910F910C942D
:103D00004D05802FDF91CF911F910F910C943D05B0
:103D1000DF91CF911F910F9108950F939C01CB01DB
:103D2000243F4CE5340731F188F4293DFCE53F0799
:103D3000D9F02A3D4CE5340779F1283D3C45A9F5F9
:103D400006E221EE41EE68ED7CE52BC0263FFCE566
:103D50003F07E1F0A8F0273F3C4539F507E225EEA3
:103D600046EE67EF7CE51DC007E225EE45EE69ED06
:103D70007CE517C006E221EE40EE64EF7CE511C061
:103D800007E225EE44EE65EF7CE50BC006E221EE8E
:103D900042EE66EF7CE505C008E221E045EE6AED03
:103DA0007CE50E941A1E80E008C0FC018281882305
:103DB00019F01092710201C081E00F910895909363
:103DC000C1018093C0010895909377028093760299
:103DD0000895E0917602F0917702309721F00190FA
:103DE000F081E02D099480E00895E0917602F09151
:103DF0007702309721F00280F381E02D0994089535
:103E000020917402309175022817390771F0909350
:103E1000750280937402E0917602F09177023097F8
:103E200021F00680F781E02D099408952091720217
:103E3000309173022817390771F0909373028093C1
:103E40007202E0917602F0917702309721F00084BF
:103E5000F185E02D09940895FC01329697E080E009
:103E6000915029F021912223D9F38F5FF9CF089542
:103E7000662349F0FC01329608962191621729F0D9
:103E8000E817F907D1F780E0089581E008959C01D3
:103E9000FC0132969FEF80E04191461789F09F3FE9
:103EA00019F4411101C0982F8F5F8630A9F79F3F09
:103EB00039F0F901E90FF11D97FDFA956283089534
:103EC00008959C012A5F3F4FFC014281461301C0C7
:103ED0001282019682179307B9F708950C94471F31
:103EE0000C94611F029626E0FC0111922A95E9F7D5
:103EF000089508950C94791F83E0809378020C94C0
:103F00007A1F811102C081E001C082E080937802B3
:103F10000C947A1F0C94811F81E0809378020C949A
:103F20007A1F0C948C1F08950C94931F0C94941F6B
:103F30000C94931F0C94931F0C94931FCF930E9487
:103F40009A1F0E94BA120E94981FC0E08C2F0E94F4
:103F5000E411892B29F4CF5FC530C1F780E001C09F
:103F600081E0CF91089508951F920F920FB60F929E
:103F700011248F939F93AF93BF9380917902811106
:103F800013C08091B5029091B602A091B702B09192
:103F9000B8024196A11DB11D8093B5029093B6025F
:103FA000A093B702B093B802BF91AF919F918F9148
:103FB0000F900FBE0F901F9018958091BD02843016
:103FC00031F10E9494031092790220E488E190E09C
:103FD0000FB6F894A895809360000FBE2093600000
:103FE00083B7817F846083BF83B7816083BF789408
:103FF000889583B78E7F83BF0FB6F894A89580917C
:104000006000886180936000109260000FBE089588
:104010000E94DA070C949D0382E084BD93E095BD75
:104020009AEF97BD80936E0008952FB7F894809112
:10403000B5029091B602A091B702B091B8022FBF1D
:1040400008952FB7F8946091B5027091B6028091EF
:10405000B7029091B8022FBF08959C014FB7F89412
:104060008091B5029091B602A091B702B091B802CA
:104070004FBF821B930B089578941F920F920FB637
:104080000F9211248F939F93AF93BF938091B502AA
:104090009091B602A091B702B091B8020196A11D0D
:1040A000B11D8093B5029093B602A093B702B0936E
:1040B000B802BF91AF919F918F910F900FBE0F905B
:1040C0001F90189581E08093E00080E28093D800F3
:1040D0001092C9008FE19EE40197F1F700C0000043
:1040E00087E090EBDC018093C6029093C702A09317
:1040F000C802B093C9029CE088E10FB6F894A89575
:10410000809360000FBE90936000FFCF8091850286
:1041100008950895CF93DF9321E02093E9002FEFD6
:104120003091E800215035FD06C035ED3A95F1F7A4
:1041300000002111F5CF2091E80025FF14C0EC010B
:1041400040E050E068E070E00E9496228091E80034
:104150008E778093E80088E0FE01ADE7B2E0019041
:104160000D928A95E1F7DF91CF91089580937A02BD
:1041700070937C0260937B028091BD02843001F5D4
:1041800082E08093E9008FEF9091E800815095FDE7
:1041900006C095ED9A95F1F700008111F5CF809159
:1041A000E80085FF0DC040E050E063E070E08AE782
:1041B00092E00E9496228091E8008E778093E8003A
:1041C0000895BC0184E00C94B620BC0183E00C94FB
:1041D000B62008958091BC02811109C00E94272455
:1041E0000E9484248091E20084608093E20008951C
:1041F0001092BC0208950C94911F6091B90281E065
:10420000611101C080E00C947C1F9091BD0281E09F
:10421000943009F080E06091B9020C94811F42E073
:1042200061EC81E00E94A02342E261EC82E00E9406
:10423000A0239091BD0281E0943009F080E060916C
:10424000B9020C948A1F8091BF02833009F461C0C7
:1042500030F4813071F0823009F49AC008958A30C8
:1042600009F486C08B3009F46CC0893009F0A8C00D
:1042700020C08091BE02813A09F0A2C08091E8007E
:10428000877F8093E8008091C2029091C302892BBE
:1042900021F468E08DE792E003C060E080E090E008
:1042A00070E00E94E1228091E8008B778093E80023
:1042B00008958091BE02813209F082C08091C202CD
:1042C0009091C302029708F07BC08091E800877F3D
:1042D0008093E8008091E80082FD05C08091BD02D6
:1042E0008111F8CF6DC02091F3008091F20090E031
:1042F000922B029731F48091F100813011F08630D9
:1043000021F48091F100809385028091E8008B7701
:1043100053C08091BE02813A09F052C08091C2021E
:104320009091C302892B09F04BC08091E800877FF0
:104330008093E8008091E80080FFFCCF809123010A
:1043400036C08091BE028132D9F58091C20290912F
:10435000C302892BA9F58091E800877F8093E8004C
:104360000E94D5238091C002809323010C94DA0728
:104370008091BE02813221F58091E800877F809391
:10438000E8000E94D5238091C1028093860208959F
:104390008091BE02813AA1F48091E800877F8093EA
:1043A000E8008091E80080FFFCCF80918602809336
:1043B000F1008091E8008E778093E8000C94D5237B
:1043C000089584B7877F84BF0FB6F894A89580912D
:1043D0006000886180936000109260000FBE90E0E2
:1043E00080E80FB6F89480936100909361000FBE4F
:1043F0000C948C1F0E9427240E948424E2EEF0E09B
:1044000080818460808378940C94192787E191E0FF
:104410000C94E41E8091BD028530A9F48091BD0208
:10442000853079F40E94DD1F8091BB028823B1F3AF
:104430000E949E1F882391F30E9480220E94DA0727
:10444000EDCF0C940820089508950C942722292F6D
:10445000332723303105C9F060F42130310581F074
:104460002230310509F044C08BE390E029E634E0C6
:1044700043C021323105E1F02232310549F138C023
:1044800082E190E024EA34E037C099278130910539
:1044900049F028F0029761F5EFE2F4E005C0E5E6A7
:1044A000F4E002C0E3E5F4E0849190E09F0124C0D1
:1044B0006115710541F061307105D1F489E090E03A
:1044C00024E934E019C089E090E02BE734E014C01F
:1044D0006115710541F06130710551F482E390E09E
:1044E00026EB34E009C080E490E028EE34E004C01C
:1044F00080E090E020E030E0FA01318320830895ED
:1045000080E189BD82E189BD09B400FEFDCF8091C3
:10451000D8008F7D8093D8008091E00082608093E6
:10452000E0008091E00081FDFCCF0895CF92DF9202
:10453000EF92FF920F931F93CF93DF93EC018B01C8
:104540007A010E94F423811133C0E114F10439F09F
:10455000F70180819181081B190BC80FD91FC12C4D
:10456000D12C0115110519F18091E80085FD16C0C7
:104570008091E8008E778093E800E114F10449F01F
:10458000F70180819181C80ED91ED182C08285E059
:104590000FC00E94F423882321F30AC089918093DD
:1045A000F10001501109FFEFCF1ADF0ADACF80E0E6
:1045B000DF91CF911F910F91FF90EF90DF90CF90FF
:1045C00008952091C4023091C5022617370748F09C
:1045D0006115710539F42091E8002E772093E800E9
:1045E00001C0B901FC0120E06115710579F18091EC
:1045F000BD028823F1F18530F1F18091E80083FD5F
:104600003CC08091E80082FD2EC08091E80080FFD0
:10461000EBCF2091F3008091F20090E0922B611596
:10462000710551F08830910538F421912093F10003
:10463000615071090196F3CF21E0089709F020E05D
:104640008091E8008E778093E800CECF2111CFCF04
:104650000AC08091BD02882361F0853061F08091AD
:10466000E80083FD0AC08091E80082FFF2CF80E07D
:10467000089582E0089583E0089581E008952091EF
:10468000C4023091C5022617370748F0611571053D
:1046900039F42091E8002E772093E80001C0B90199
:1046A000FC0120E06115710591F18091BD02882324
:1046B00009F440C0853009F43FC08091E80083FDD3
:1046C0003DC08091E80082FD2FC08091E80080FF0E
:1046D000E9CF2091F3008091F20090E0922B6115D8
:1046E000710559F08830910540F424912093F10030
:1046F0003196615071090196F2CF21E0089709F0D7
:1047000020E08091E8008E778093E800CBCF2111E4
:10471000CCCF0AC08091BD02882361F0853061F062
:104720008091E80083FD0AC08091E80082FFF2CF0B
:1047300080E0089582E0089583E0089581E008957F
:10474000982F973068F59093E900981739F0709199
:10475000EC002091ED005091F00003C0242F762F43
:1047600050E021FD02C09F5FECCF3091EB003E7F17
:104770003093EB003091ED003D7F3093ED003091B0
:10478000EB0031603093EB007093EC002093ED0070
:104790005093F0002091EE0027FDE5CF80E00895D2
:1047A0008F708093E90081E008958091BE0287FFB9
:1047B00011C08091E80082FD05C08091BD02811189
:1047C000F8CF11C08091E8008B770BC08091BD02BB
:1047D000882349F08091E80080FFF8CF8091E800BD
:1047E0008E778093E80008952091E4003091E500F1
:1047F00095E64091EC00842F817040FF23C08091AA
:10480000E80080FD1DC08091BD02882399F08530AD
:1048100099F08091EB0085FD11C04091E40050912A
:10482000E5002417350729F3915011F09A01E1CFE3
:1048300084E0089582E0089583E0089581E008957A
:1048400080E008954091E80042FFDDCF08950E9486
:1048500095240E949D24E0EEF0E0808181608083B9
:10486000E8EDF0E080818F77808319BCA7EDB0E0A0
:104870008C918E7F8C9380818F7E80831092BC027E
:1048800008950F931F93CF93DF930E9495240E9466
:104890009D24C8EDD0E088818F77888388818068E7
:1048A000888388818F7D888319BC1092BD02109205
:1048B000B9021092BB021092BA0200EE10E0F801A9
:1048C00080818B7F808388818160888342E060E083
:1048D00080E00E94A023E1EEF0E080818E7F808363
:1048E000E2EEF0E080818160808380818860808357
:1048F000F80180818E7F8083888180618883DF9149
:10490000CF911F910F910895E8EDF0E080818F7EA7
:104910008083E7EDF0E080818160808384E082BF66
:1049200081E08093BC020C944124E8EDF0E08081AA
:104930008E7F80831092E20008951092DA00109228
:10494000E10008951F920F920FB60F9211242F933A
:104950003F934F935F936F937F938F939F93AF9307
:10496000BF93EF93FF938091E10082FF0BC0809192
:10497000E20082FF07C08091E1008B7F8093E1001D
:104980000E9418278091DA0080FF1FC08091D80014
:1049900080FF1BC08091DA008E7F8093DA008091C7
:1049A000D90080FF0DC080E189BD82E189BD09B4D5
:1049B00000FEFDCF81E08093BD020E94EA2005C089
:1049C00019BC1092BD020E94F8208091E10080FF86
:1049D00019C08091E20080FF15C08091E2008E7FB7
:1049E0008093E2008091E20080618093E2008091F8
:1049F000D80080628093D80019BC85E08093BD0206
:104A00000E94FD208091E10084FF30C08091E2008F
:104A100084FF2CC080E189BD82E189BD09B400FE1C
:104A2000FDCF8091D8008F7D8093D8008091E100E8
:104A30008F7E8093E1008091E2008F7E8093E20080
:104A40008091E20081608093E2008091B902882326
:104A500011F084E007C08091E30087FD02C081E08F
:104A600001C083E08093BD020E9405218091E10096
:104A700083FF29C08091E20083FF25C08091E1007F
:104A8000877F8093E10082E08093BD021092B9029B
:104A90008091E1008E7F8093E1008091E2008E7F23
:104AA0008093E2008091E20080618093E20042E026
:104AB00060E080E00E94A0238091F00088608093F5
:104AC000F0000E94FB20FF91EF91BF91AF919F9169
:104AD0008F917F916F915F914F913F912F910F90A7
:104AE0000FBE0F901F9018951F920F920FB60F9246
:104AF00011242F933F934F935F936F937F938F93E3
:104B00009F93AF93BF93CF93DF93EF93FF93C091A6
:104B1000E900CF708091EC00D82FD17080FDD0E8F3
:104B20001092E9008091F000877F8093F0007894E4
:104B30000E94B8251092E9008091F000886080936F
:104B4000F000CD2BCF70C093E900FF91EF91DF9182
:104B5000CF91BF91AF919F918F917F916F915F9115
:104B60004F913F912F910F900FBE0F901F9018956E
:104B70001F93CF93DF93CDB7DEB7AA970FB6F89404
:104B8000DEBF0FBECDBFEEEBF2E08091F10081936E
:104B900022E0E63CF207C9F70E9423218091E80059
:104BA00083FF2EC18091BE029091BF02492F50E039
:104BB0004A30510508F024C1FA01EE59FF4F0C9418
:104BC0009C27803821F0823809F01AC108C08091F2
:104BD000BA029091BB02992389F082600FC0809144
:104BE000C2028F70873008F00BC18093E90080917A
:104BF000EB0085FB882780F91092E9009091E8008E
:104C0000977F9093E8008093F1001092F100D1C05B
:104C1000282F2D7F09F0F4C0882319F0823061F02D
:104C2000EFC08091C002813009F0EAC0933009F0F2
:104C300080E08093BB022EC08091C00281112AC007
:104C40008091C2028F702FEF280F263008F0D8C055
:104C50008093E9002091EB0020FF1CC0933021F4E9
:104C60008091EB00806214C09091EB009061909372
:104C7000EB0021E030E0A90102C0440F551F8A95E6
:104C8000E2F74093EA001092EA008091EB0088601E
:104C90008093EB001092E9008091E800877F809379
:104CA000E8000E94D523ACC08111AAC01091C002B7
:104CB0001F778091E3008078812B8093E3008091BF
:104CC000E800877F8093E8000E94D5238091E80068
:104CD00080FFFCCF8091E30080688093E300111196
:104CE00002C082E001C083E08093BD0289C0805889
:104CF000823008F085C08091C0029091C1028C3D45
:104D000053E0950779F583E08A838AE289834FB778
:104D1000F894DE01139620E03EE051E2E32FF0E04C
:104D200050935700E49120FF03C0E295EF703F5F7E
:104D3000EF708E2F90E0EA3010F0C79601C0C09659
:104D40008D939D932F5F243149F74FBF8091E800E9
:104D5000877F8093E8006AE270E0CE0101960E94AE
:104D6000E12216C06091C2027091C302AE014F5F92
:104D70005F4F0E942522BC01892B09F441C090910C
:104D8000E800977F9093E80089819A810E943F23F1
:104D90008091E8008B778093E80032C0803881F5FD
:104DA0008091E800877F8093E8008091B90280932A
:104DB000F1008091E8008E7772CF811121C080913F
:104DC000C0029091C10299270297D4F48091E80023
:104DD000877F8093E8008091C0028093B9020E948F
:104DE000D5238091B902811106C08091E30087FD2F
:104DF00002C081E001C084E08093BD020E940F21C7
:104E00008091E80083FF0AC08091E800877F80934B
:104E1000E8008091EB0080628093EB00AA960FB6C9
:104E2000F894DEBF0FBECDBFDF91CF911F910895E3
:104E30000895CF938091BD028823A1F0C091E9002D
:104E4000CF709091EC00892F817090FD80E8C82B85
:104E50001092E9008091E80083FD0E94B825CF7090
:104E6000C093E900CF910895DB018F939F930E9437
:104E7000C027BF91AF91A29F800D911DA39F900D60
:104E8000B29F900D1124089587FB082E062687FDFA
:104E9000819567FD61950E94D3270EF4919507FCDB
:104EA00081950895AA1BBB1B51E107C0AA1FBB1F18
:104EB000A617B70710F0A61BB70B881F991F5A95A6
:104EC000A9F780959095BC01CD01089597FB072E19
:104ED00016F4009407D077FD09D00E94522707FCF2
:104EE00005D03EF4909581959F4F089570956195FA
:104EF0007F4F0895A1E21A2EAA1BBB1BFD010DC016
:104F0000AA1FBB1FEE1FFF1FA217B307E407F50779
:104F100020F0A21BB30BE40BF50B661F771F881F55
:104F2000991F1A9469F760957095809590959B01EB
:104F3000AC01BD01CF010895EE0FFF1F0590F49164
:104F4000E02D09940E94AA27332312F48A1B9B0B9D
:104F50000C94BB27A29FB001B39FC001A39F700D0B
:104F6000811D1124911DB29F700D811D1124911D71
:104F700008950E94AA27B7FF0895821B930B0895F6
:104F80000E94AA27A59F900DB49F900DA49F800D0D
:104F9000911D11240895B7FF0C94C0270E94C027CB
:104FA000821B930B0895991B79E004C0991F9617F3
:104FB00008F0961B881F7A95C9F780950895FC0123
:104FC0004150504030F001900616D1F73197CF0193
:104FD0000895882799270895FB01DC0104C08D916D
:104FE0000190801921F441505040C8F7881B990B5B
:104FF0000895F999FECF92BD81BDF89A992780B5A1
:105000000895A6E1B0E044E050E00C943328A8E114
:10501000B0E042E050E00C943328262FF999FECFFF
:1050200092BD81BDF89A019700B4021639F01FBAFB
:1050300020BD0FB6F894FA9AF99A0FBE0895039618
:10504000272F0E940E280E940D28252F0E940E282F
:10505000242F0C940E280196272F0E940E280C94C2
:105060000D28DC01CB01FC01F999FECF06C0F2BD91
:10507000E1BDF89A319600B40D9241505040B8F716
:065080000895F894FFCF33
:10508600C8004002010102000600060601191A1BAB
:105096001C1D1E1F20212286208A20E920E520E1F2
:1050A60020892001E200E900EA00B500B600B70059
:1050B600CD008301CC008A019201940121022302D2
:1050C60024022502260227022A02B300B4006F003A
:1050D6007000818283E200E900EA00B500B600B7FD
:1050E60000CD008301CC008A0192019401210223A4
:1050F6000224022502260227022A02B300B4006F08
:1051060000700081828331F5F6F76766363534978D
:105116009694959392309091F0F4F1000102020278
:10512600020606060909090909090F0F0F0F0F0FD5
:1051360015151518191919191919191919192324D1
:00000001FF
